:020000000C945E
:1000020038000C9400000C9400000C9400000C9436
:1000120000000C9400000C9400000C9400000C945E
:1000220000000C9400000C94C8010C9400000C9485
:10003200B5030C9468000C9400000C94DA000C9444
:1000420000000C9400000C9400000C9400000C942E
:1000520000001027E80364000A00010000100001FC
:100062001000010000000200DF0266000000F894A8
:10007200EE27ECBBF1E0FBBFEBBFE5BFF8E1F1BD62
:10008200E1BD8DE0A2E0BB27ED938A95E9F780E020
:1000920098E0A0E6ED930197E9F7E8E6F0E08591B4
:1000A2009591009761F0A591B59105901590BF01CA
:1000B200F00105900D920197E1F7FB01F0CFEFE51A
:1000C200EDBFE8E0EEBFC0E6D2E00C949402AA9342
:1000D200EA93FA93EFB7EA931A930A93AF93BF9313
:1000E200EF93FF93AFB7AF931BB10CB1E12FEC715C
:1000F20009F5E0919102F0E0E758FD4F0083A091ED
:100102009102AF5FA0939102A83119F4E0E0E0936D
:100112009102A0919302AF5FA0939302A83129F4B8
:10012200E0E0E0939302689420F8442009F4DE9A18
:10013200EAE04E2EAF91AFBFFF91EF91BF91AF9129
:1001420009911991E991EFBFF991E991A991189556
:100152001A9388249924E0919302E03049F4E4E66A
:10016200F0E08E169F061CF0E0E019910895F3CF9F
:10017200E0919202F0E0E758FD4F1081A0919202C7
:10018200AF5FA0939202A83119F4E0E0E0939202EB
:10019200F894E0919302E150E09393027894E12F76
:1001A20019910895A0919302E0E00E94AE0DF0E053
:1001B2000895AA93EA93FA93EFB7EA93AF93BF93A2
:1001C200EF93FF93AFB7AF93E091B202E030C9F083
:1001D200E150E093B202E091B102F0E0E856FD4F47
:1001E200E081ECB9A091B102AF5FA093B102A83156
:1001F20019F4E0E0E093B102442009F4DE9AEAE067
:100202004E2EAF91AFBFFF91EF91BF91AF91E991A8
:10021200EFBFF991E991A9911895A091B202A83185
:10022200E1F35D9BFECFF894E091B202E03011F46D
:100232005D9917C0E091B002F0E0E856FD4FA88149
:10024200A083A091B002AF5FA093B002A83119F4CD
:10025200E0E0E093B002E091B202EF5FE093B2021D
:1002620002C0E881ECB9789421960895E091D60213
:10027200F091D7023196E093D602F093D702E09143
:100282006002E03099F0B29902C00E943C0CE09109
:100292007102E03011F00E943C0C0E94420C2CF0E2
:1002A2000E943C0CE3E0E093750228C00E94420CDD
:1002B2002CF00E943C0CE5E0E0937402E0917202A3
:1002C200E03011F066247724F30131963F01E8E52E
:1002D200F2E0E615F70530F466247724E3E0EA93CA
:1002E2000E94E904A091B302AF5FA093B302A230CF
:1002F20029F4E0E0E093B3020E944A090895E091F4
:100302006002E03011F00E949B080E9465080E9482
:100312008408A0916302A13028F0E0916302E150C9
:10032200E093630208950E94AA07F40131964F01F7
:10033200E0919402F09195023196E0939402F09349
:100342009502A0919402B09195021A9744F0E0E0D0
:10035200E0939402E09395020E94800101C0089507
:10036200E0919602F09197023196E0939602F09313
:100372009702A0919602B09197021A973CF0E0E0A2
:10038200E0939602E09397020E94370108950E943B
:100392004A0CAF93BF93EF93FF93AFB7AF93E09144
:1003A200B502EF5FE093B502E13039F4ECB7E15EFC
:1003B200ECBF0E94B90A0C942F02E23059F4ECB758
:1003C200E15EECBFE1E0EA930E94B70B0E94B90A3A
:1003D2000C942F02E33039F4ECB7E15EECBF0E94DB
:1003E200B90A0C942F02E43059F4ECB7E05EECBF8A
:1003F200E0E0E093B502EA930E94B70B0E94B90ACB
:10040200F50131965F01E8E0F0E0AE16BF062CF090
:10041200AA24BB240E94F00A02C00C942F02F60107
:1004220031966F01EAE0F0E0CE16DF06BCF0CC2494
:10043200DD240E94CF0B442019F04A9409F4DE987F
:10044200E091B402E03051F4E1E0E093B402789438
:100452000E949401F894E0E0E093B402AF91AFBF40
:10046200FF91EF91BF91AF910E94580C1895B399EB
:1004720058C0F894E0E0EBBBE5BB859904C0DD9A77
:10048200A8950C943E02849904C0DC9AA8950C9419
:100492004402879904C0DF9AA8950C944A0286996F
:1004A20004C0DE9AA8950C945002829904C0A89ABE
:1004B200A8950C945602B59904C0DB9AA8950C94A1
:1004C2005C02B49904C0D99AA8950C946202B799B7
:1004D20004C0DA9AA8950C946802B69904C0D89A16
:1004E200A8950C946E02839905C0DB9AD89AA895B8
:1004F2000C947402B09905C0DA9AD99AA8950C9412
:100502007B02B19905C0DB9AD89AA8950C94820215
:10051200B29905C0DA9AD99AA8950C9489020C94DA
:10052200380278940895E0E0EBBBEFEFEABBE8BB5A
:10053200E0E0E7BBE2E0E5BBE1ECE4BBE0E0E2BB2C
:10054200E1BBE2E0E3BFE0E0E2BFE4E6ECBFE0E013
:10055200EFBDEEBDEDBDECBDEBBDEABDE9BDE8BD55
:10056200E2BDE5BDE4BDE3BDEBB7EBBFE0E0E5BF57
:10057200E4BFE2E0E9BFE0E0EBB9E8EDEAB9E6E8C2
:10058200E0BDE0E0E0BDE9E1E9B9E0E8E8B9E0E0DA
:10059200E0BFE1E0E0936002E0E0E0937102E0930B
:1005A2007202E0E0E0939602E0939702E0E0E093CB
:1005B2009402E0939502CC24DD24AA24BB2488244F
:1005C2009924E0E0E0936102E0936202E093630227
:1005D200E0E0E0936902E0936A020E94660C55240F
:1005E2000E946C0CE8E6F1E00E94720CE0E0E093FD
:1005F2007002E0936F02E09366020E94770C662419
:100602007724E0E0E0937302E0937502E0937602D0
:10061200E4E0E0937402E0E0E0937702E1E0E0934B
:1006220078020E94F8090E9410070E94BC030E94EF
:100632007D0CE23020F00E947D0CE93130F0A8956B
:10064200ECE0A1E0B0E00E94040E7894A8986297D2
:10065200E6B3E170A0E00E94A90DE0936002A895C4
:10066200B39902C00E943802E0916002E030E1F1E9
:100672000E94D3003097B9F1A89A0E94820C19F017
:1006820062960C9428030E948A0C18F0AF85AA3057
:1006920018F062960C9428030E94930C0E949D0C01
:1006A200ACF40E94A50CEA0FFB1FFF93EF930E948C
:1006B200A900AF91BF91EC930E94A50C0E94AA0CD5
:1006C200E881F9813196E883F983E8CFEE85E0305D
:1006D20019F062960C9428030E94B10C0E949E06A7
:1006E2000E943C0CA8983CC00E94D3003097C1F1F4
:1006F2000E94820C19F062960C9428030E948A0CC4
:1007020018F0AF85AA3018F062960C9428030E9464
:10071200930C0E949D0CACF40E94A50CEA0FFB1FE7
:10072200FF93EF930E94A900AF91BF91EC930E94B7
:10073200A50C0E94AA0CE881F9813196E883F9831D
:10074200E8CFEE85E03019F062960C9428030E94FF
:10075200B10C0E94860566247724E0E0E0937202E1
:1007620062960C942803FFCF0E944A0C0E949402C6
:100772000E94580C1895E0E0E093B602E093B702AD
:10078200E0E0E093B802E0E0E093B902E093BA025D
:10079200E0E0E093BB0208950E94150EEF81E0684D
:1007A200EF83EE81EE5FEE8330E0E1E0EA930E94B8
:1007B2000E01EE81EA930E940E01EE813E0FEF815F
:1007C200EA930E940E01EF813E0F00E010E0EE81FD
:1007D200E250D801F0E0AE17BF075CF40E94BA0CF9
:1007E200EA930E940E010E94BA0C3E0F0F5F1F4F48
:1007F200EECFE32FF0E0A0E0B1E00E94F10DEA1BA2
:100802003E2F3A930E940E0186C2E0917402A881A3
:10081200B981EC93E0916102E03069F41196E1E074
:10082200EC93E0917002E03029F0A881B981119631
:10083200E4E0EC931CC0E33011F0E13009F412C0A3
:10084200E23029F4A881B9811196E3E00FC0E430C7
:1008520071F4A091B802A23029F4A881B98111964D
:10086200E3E004C0A881B9811196E2E0EC93E09143
:100872006502E03029F0A881B9811196E5E0EC9398
:100882000E94C10C0E94A40DA881B9811296EC931A
:100892000E94C10CF070A881B9811396EC93E0918B
:1008A200B602F091B7020E94A40DA881B9811496F4
:1008B200EC93E091B602F091B702F070A881B98191
:1008C2001596EC93E881F9813696A0917802A0837F
:1008D200EA81EA93E7E00E94C60C78C01A93E0919D
:1008E2007302E03011F410E017C0E13011F0E23091
:1008F20011F411E011C0E33011F412E00DC0E43044
:1009020011F0E53011F413E007C0E63011F414E001
:1009120003C0E73009F417E0A981BA811C9311964C
:100922000E94CD0C12960E94CD0C13960E94CD0C03
:1009320014960E94CD0C15960E94CD0C1696E0E0FE
:10094200EC93EB81EA93E7E0EA93EB81FC810E946E
:10095200D20C188124960895E091BB02E03011F088
:10096200E0E00895E0E0E093B602E093B7020E946F
:10097200D60CD99AE3E0E0936102E1E008950E9487
:10098200DD0C0895E091BB02E03011F0E0E01EC002
:10099200E881F981E0936902F0936A020E94E50C12
:1009A200EA17FB0741F4E0916102E03011F00E9486
:1009B200DD0CE1E00BC0EA81E03019F0D99AE2E007
:1009C20002C0D89AE1E0E0936102E1E02396089543
:1009D2000E94130EE0E0E0937102E0937702EE8151
:1009E200E13011F0E23059F4A0917402A23009F41E
:1009F20088C0E091BE02E03009F083C01DC0E33040
:100A020031F4E0917402E03009F47BC015C0E730A4
:100A120099F4E0917602E43011F0E53009F402C075
:100A2200E63031F4E7E0E09376020E94EA0C69C016
:100A3200E7E0E093760265C0A091BF02A13011F019
:100A42000C947405EE81E13011F4E4E007C0E23069
:100A520011F4E5E003C0E33011F4E6E0EE83009127
:100A6200B9021091BA02005010402CF00E94F10C11
:100A72000E171F0714F000E010E00E94E50CF801C9
:100A8200EA1BFB0B9F010E94F60CE2E0F0E00E94E1
:100A9200DE0DE217F30724F40E94F60C2A1B3B0B2F
:100AA2000E94F10C0E94A00DDF01E2E0F0E00E9442
:100AB200DE0D2E173F0724F40E94F10C2E0F3F1F6C
:100AC200D901E0E0F0E00E94B80D5E2FE0E0E09393
:100AD200BB025A931A930A930E94C304E1E0E09383
:100AE200BB02EE810CC0EE81E13011F4E1E007C0FF
:100AF200E23011F4E2E003C0E33019F4E3E0E09302
:100B020076020E941A0E279608950E94150EEF8112
:100B1200EA3059F4AE81A23009F0FDC0AC81BD814A
:100B2200E6E00E94FB0C0C949A06E33069F4AE8175
:100B3200A23009F0F0C00E94C0040E94030DE0E060
:100B4200E09370020C949A06E43079F4AE81A230FC
:100B520009F0E1C0E0E0E09370020E94AD04AC81D4
:100B6200BD810E94FB0C0C949A06E530C9F5AE815A
:100B7200A53009F0D0C00E940A0D28F0AC81BD81D9
:100B8200AC91A33008F0C7C0AC81BD81AC91E1E06B
:100B92000E94A90D1E2FAC81BD8111962C91332785
:100BA200322F2227AC81BD8112960E940F0D2E0F8B
:100BB2003F1F205030402CF00E94F10C2E173F07AF
:100BC2000CF0A9C0E0E0E09370021A933A932A93E2
:100BD2000E94C304AC81BD810E94FB0C0C949A0656
:100BE200E63019F5AE81A33009F095C00E940A0DD6
:100BF20079F0AC81BD81AC91A33051F0AC81BD8163
:100C0200AC91A23029F0AC81BD81AC91A73059F4EE
:100C1200E0E0E0937002AC81BD81EC91EA930E9426
:100C2200E9040E94030D0C949A06E73071F4AE8138
:100C3200A23009F070C0EF81EA93ED81FE81FA9350
:100C4200EA930E9406040C949A06E83069F4AE8195
:100C5200A23009F060C00E946C0CE0E0E0937002E8
:100C62000E94030D0C949A06E93019F5AE81A43066
:100C720009F051C0AC81BD810E940F0D0E94720C1F
:100C8200F0916D02E0E00E94720CAC81BD81119680
:100C9200EC910E94F60CF0E0EA0FFB1F0E94720C2E
:100CA200E0E0E0937802E09370020E94030D0C945E
:100CB2009A06EB3059F5AE81A53069F5AC81BD815C
:100CC200AC91A03019F00E940A0DF1F4AC81BD8103
:100CD200EC91E093BF0211960E940F0D0E94120D3B
:100CE200F091B902E0E00E94120DAC81BD81129632
:100CF200EC91A091B902B091BA02F0E0EA0FFB1FA9
:100D02000E94120D0E94030D0C949A06EC3089F495
:100D1200AE81A33021F00E941C0E28960895A8955A
:100D2200AC81BD81EC91A1E0B0E00E94040E0E9472
:100D3200030D0E941C0E28960895EB81EA3071F48F
:100D4200AA81A23009F042C0A881B981E6E8EC93F9
:100D5200EB81EA93E1E00E94C60C38C0E33051F423
:100D6200AA81A23099F5E7E00E94170DE0E0E09336
:100D720070022CC0E630E9F4AA81A33039F5A881CB
:100D8200B981AC91A13079F0A881B981AC91A3303D
:100D920051F0A881B981AC91A23029F0A881B98122
:100DA200AC91A73029F4A881B981EC910E94170D6A
:100DB2000DC0E73059F4AA81A23041F4EB81EA93E5
:100DC200E981FA81FA93EA930E946F0424960895C6
:100DD2001A93E0B3E07F1E2FE12FE071A0E00E94A2
:100DE200AE0DAF81B885EC93E12FE072A0E00E94D6
:100DF200AE0DAB81BC81EC93E12FE074A0E00E94C8
:100E0200AE0DAD81BE81EC93E12FE078A0E00E94AF
:100E1200AE0DA981BA81EC93188129960895E0E07C
:100E2200E093BC02E093BD02E093BE02E093BF02F6
:100E320008950E94660CE0916F02E03081F1E0E0DB
:100E4200E0936F02E1E0E09370020E94C10CE09334
:100E5200B602F093B7020E946C0CA0916102A2301C
:100E620081F40E94F10CA3E0B0E00E94C60DDF0104
:100E72000E941E0DEA17FB071CF4E4E0E0936102F6
:100E82000EC0A0916102A13051F40E94F60C0E94A2
:100E92001E0DAE17BF071CF4E4E0E0936102E0917F
:100EA2006102E13081F40E94270D24F40E94300D8A
:100EB2000E94320D0E94390D29F40E94EA0CE1E0F1
:100EC200E093620245C0E23079F40E94470D0E942D
:100ED200300DAE17BF0714F00E944E0D0E94390D5F
:100EE20011F40E94EA0C34C0E33091F4E0E0E093A4
:100EF2006202EFE0E0936302E0917002E03029F0D9
:100F02000E946C0C0E94EA0C02C00E94470D20C095
:100F1200E43019F40E94EA0C1BC0E030C9F4A0913D
:100F22006302A130A8F0E0916202E03041F00E9439
:100F3200270D24F40E94300D0E94320D09C00E9438
:100F4200470D0E94300DAE17BF0714F00E944E0DE0
:100F520008950E94150EE0916002E03011F00C94A9
:100F6200F907E0B3E470A0E00E94A90D0E2F003053
:100F720011F0DD9A01C0DD98E0917002E03031F4A9
:100F8200E0916F02E03011F4003009F40FC0E091FB
:100F92006602EF5FE0936602A0916602A33030F032
:100FA200E0E0E0936602E1E0E0936F02E0B3E87014
:100FB200A0E00E94A90D1E2FA091BC021A17B9F041
:100FC20053940E947D0CE51588F455241093BC02BD
:100FD2000E941A07EBB3EF7EAE2FE091BC02E03025
:100FE20011F0E0E101C0E0E0EA2BEBBB01C05524C7
:100FF200E6B3E07C3E2FE32FE095E07C3E2F3030DD
:1010020019F0E0E0E0936402A09168023A1711F44B
:101012000C946408E0916002E03029F1303029F04C
:10102200E0916802E32BE03C69F40E94570DA53180
:1010320040F00E94770CE7E0E0937502E1E0E09374
:10104200710210C00E94570DA73460F00E945F0D1C
:10105200303411F4E3E001C0E1E0E0937502E1E035
:10106200E093710230C0303059F0E0916802E32B16
:10107200E03C31F0A0916102A13011F0A23061F4A4
:101082000E94570DA53138F00E94770C0E94EA0C9D
:10109200E0E0E093700217C00E94570DA73498F069
:1010A2000E945F0DE0E0E0937002303429F4E1E049
:1010B200E0936102D89A04C0E2E0E0936102D99A17
:1010C200E1E0E0937202E1C0E0916002E03009F0F9
:1010D2000895E0916102E03091F0E0916402EF5FE7
:1010E200E0936402A0916402A43641F40E94EA0CE7
:1010F200E0E0E0936402E1E0E093650203C0E0E037
:10110200E09364020895E6B3E095E073E093BE02D3
:10111200E03079F0E0916002E03039F0E091730262
:10112200E03011F00E94650D04C0E3E0EA930E94F2
:10113200E90408950E94150EEDB7FEB7FA93EA93FB
:101142001F93EDB7FEB7FA93EA930F93EDB7FEB78D
:10115200FA93EA933F93EDB7FEB7FA93EA932F938C
:101162000E94E9062F913F910F911F91EBB3EF700F
:10117200EBBB303021F0EBB3ED7FE062EBBB203014
:1011820021F0EBB3E77FE068EBBB103021F0EBB36B
:10119200EE7FE061EBBB003021F0EBB3EB7FE0646C
:1011A200EBBBB19902C021E001E0E0917502E730AA
:1011B20039F4E0E0E093BD02EBB3E07FEBBB48C063
:1011C200E23061F4E1E0E093BD02103019F40E94D4
:1011D2006A0D03C0E0E0E09375023DC0E130B1F476
:1011E200E0E0E093BD02103019F40E946A0D0DC0D8
:1011F200003041F4EBB3E07FEBBBDA9AE2E0E0933C
:10120200730203C0E0E0E093750225C0E33019F5F4
:10121200E0E0E093BD02203089F4303039F0E7E0BD
:10122200E0937302EBB3E07FEBBB07C0EBB3E07F6D
:10123200EBBBDB9AE4E0E09373020DC0303041F483
:10124200EBB3E07FEBBBD99AE5E0E093730203C016
:10125200E0E0E0937502E0917502E030B1F43030E5
:1012620011F0203009F402C0E0E00DC0103039F076
:10127200003021F4E091BD02E03009F001C002C06B
:10128200E3E001C0E6E0E09373020E941C0E2496A4
:1012920008951A9310E0E0917602E03021F4E0E044
:1012A200E09377028DC0E43081F4A0917402A13002
:1012B20011F0A23009F481C0E0916102E03009F03E
:1012C2007FC0E1E0E093760202C0E13089F4A091B0
:1012D2007402A13011F0A23009F46FC00E94720DA5
:1012E20018F00E94790D6CC0E2E20E94820D68C083
:1012F200E53081F4A0917402A13011F0A23009F41A
:101302005CC0E0916102E03009F05AC0E2E0E09393
:10131200760202C0E23089F4A0917402A13011F089
:10132200A23009F44AC00E94720D18F00E94790D91
:1013320047C0E3E30E94820D43C0E63079F4A091F6
:101342007402A33011F0A03009F437C0E0916102B9
:10135200E030B1F5E3E0E093760202C0E33089F4D5
:10136200A0917402A33011F0A03009F426C00E94AB
:10137200720D18F00E94790D23C0E4E40E94820DE0
:101382001FC0E730B9F4A0917402A23021F0A0305E
:1013920011F0A43009F411C00E94720D20F0E5E0B2
:1013A200E09374020AC0E5E50E94820DE0E0E0935A
:1013B200BB0206C0E0E0E0937702E0E0E093760251
:1013C200A0917602A03039F4A0917402A03011F0FD
:1013D200A23009F401C003C0E0E0E093BB02103088
:1013E20021F4E1E1EA930E94080C199108950E9408
:1013F2003C0CE0E0E093D102E093D202E0E0E09323
:10140200D402E093D502E0E0E093D302E093D80265
:10141200E093D9020895E881E13069F4A091730262
:10142200A33021F0E091BE02E03009F003C0E1E018
:101432000E94870D23C0E23069F4A0917302A330A9
:1014420021F0E091BE02E03009F003C0E2E00E9428
:10145200870D14C0E33039F4E0917302E03011F0EB
:101462000E94650D0BC0E73041F4E0917302E03059
:1014720019F0E7E00E94870D01C078C077C00E9492
:101482003C0CE0916002E03011F40C949D0AE8817A
:10149200E13191F1E23269F4A0917302A33021F0BB
:1014A200E091BE02E03009F003C0E1E00E94870D46
:1014B20023C0E33369F4A0917302A33021F0E091D9
:1014C200BE02E03009F003C0E2E00E94870D14C0C2
:1014D200E43439F4E0917302E03011F00E94650DBA
:1014E2000BC0E53541F4E0917302E03019F0E7E01A
:1014F2000E94870D01C03AC0E0917302E03011F4FE
:10150200E3E317C0E13011F0E23011F4E2E211C07E
:10151200E33011F4E1E10DC0E43011F0E53011F4F3
:10152200E4E407C0E63011F4E5E503C0E73001F476
:10153200E6E6EA936CD11AC0E881E23211F4E1E006
:1015420013C0E43411F4E3E00FC0E13111F4E2E03E
:101552000BC0E33311F4E0E007C0E53511F4E4E039
:1015620003C0E63601F4E5E0E093740221960895A3
:101572001A93E3B3E2701E2FE091DA02E11751F4FD
:10158200A091DB02A13028F0E091DB02E150E09370
:10159200DB020CC0E091DB02ED5FE093DB02A09185
:1015A200DB02A93218F0E8E2E093DB02A091DB0251
:1015B200E4E10E94B30DE093D9021093DA02E5B39D
:1015C200EE7F0E2EE091D802A091D902EA2B11F003
:1015D200E1E001C0E0E0E029E5BB19910895AF998F
:1015E20008950E948B0D3196E093D402F093D502B8
:1015F200A091D402B091D5021A972CF0E0E0E093CA
:10160200D402E093D502E091DC02F091DD02319642
:10161200E093DC02F093DD02E091D202E030C1F50A
:10162200E091D902A091D302EA1769F1A091DC02FC
:10163200B091DD02199730F0A091DC02B091DD0289
:101642001C9708F018C0E091DE02EF5FE093DE0223
:10165200A091DE02AB3070F0E6EEE093D202E0E061
:10166200E093CE02E093DE02E5E0F0E0E093D40204
:10167200F093D50203C0E0E0E093DE02E0E0E09305
:10168200DC02E093DD02E091D902E093D3026DC067
:10169200E63E39F50E948B0D309711F50E94900DB0
:1016A20029F0E091CD02E160E093CD02A091CD025C
:1016B200A63E49F4E0E0E093CF02E093D002E2E0FC
:1016C200E093D20252C0A091CE02AF5FA093CE02AD
:1016D200A13230F0E0E0E093D202E093CE0245C0C6
:1016E20044C0E23011F00C94B50B0E948B0D309780
:1016F200D1F50E94900D29F0E091CD02E160E093D6
:10170200CD02A091D002AF5FA093D002A83058F1D1
:10171200E0E0E093D002E091CF02EF5FE093CF02EE
:10172200E150F0E0E653FD4FA091CD02A083A091DD
:10173200CF02A330C0F0E0E0E093D202E091CB020E
:10174200AAE5EA27A091CA02EA1779F4E091CC024D
:10175200A5EAEA27A091CA02EA1739F4E091CA027F
:10176200EA930E94400A01C0089508951A93E981FC
:10177200E03031F0E091D802E03011F0E1E001C058
:10178200E0E01E2FE5B3EF7BAE2F103011F0E0E466
:1017920001C0E0E0EA2BE5BB18816BC0A091D10249
:1017A200A130A0F1A23060F0E091D102E150E093CB
:1017B200D102E0E8E093C902E0E0E093C8020895B4
:1017C200E091C8020E94990DE081A091C902EA232A
:1017D200A0E00E94AE0DE093D802E091C902E69526
:1017E200E093C902E03091F4E0E8E093C902E091AD
:1017F200C802EF5FE093C802A091C802A83030F09F
:10180200E0E0E093D102AF98E093D80208951A93F2
:1018120010E00E949D0DA0E0A0830E949D0DAAEA07
:10182200A0830E949D0DAAEAA0830E949D0DA6EEB0
:10183200A0830E949D0DA981A0830E949D0D0F018E
:10184200A981EAE5EA27D001EC930E949D0D0F01E0
:10185200A981E5EAEA27D001EC930E949D0DA0E060
:10186200A083AF9AE0E0E093D802E5E1E093D102F1
:10187200188122960895E0E0E093D602E093D70221
:101882000895A091D602B091D702A935E2E0BE0731
:1018920008950A921A92FA926A937A938A939A9381
:1018A200AA93BA93EA93FA93EFB7EA930895E99168
:1018B200EFBFF991E991B991A991999189917991A2
:1018C2006991F990199009900895E0E0E09364021B
:1018D200E09365020895E0E0E0936B02E0936C020E
:1018E2000895E0936D02F0936E020895E0E0E093B4
:1018F2006702E09368020895A1E0B0E00E94F80D4B
:101902000895E0E0EE870E94A900E98BA989A13041
:1019120008950E94A900EF87AE85EA0FEE87AF8592
:10192200A13008950E94A900E88BAE85EA0FEE87E8
:10193200E0E0E883E9830895EF85E150A881B98169
:10194200F0E0AE17BF070895E881F981DE01129633
:101952000895AE0FBF1FEC91AE85EA0FEE87089592
:10196200E889EA93E889EA93FE013496FA93EA93C6
:101972000895F801AC81BD81AE0FBF1FEC910895AF
:10198200E0916B02F0916C020895EA93EA81FB8187
:10199200FA93EA930C94CD03E0E0EC93A981BA8127
:1019A2000895FA93EA930C94CD03EFEFFFEFE093DF
:1019B2006902F0936A020895E0916102E093B8022D
:1019C200E4E0E09361020895A0916B02B0916C0291
:1019D2000895E0E0E0936102EBB3EC7FEBBB089586
:1019E200E0916D02F0916E020895A0916D02B091A6
:1019F2006E020895EC93EF81EA93E1E0EA93EE81BF
:101A0200FF81CFCFEF81EA93E0E0EA93EE81FF819D
:101A1200C8CFAC81BD81AC91A1300895EC91F0E0CA
:101A22000895E093B902F093BA020895EA930E94EE
:101A32000C0AEB81EA93E0E0A8CFE4E0F0E00E9438
:101A4200DE0DA0916902B0916A02089599DF319783
:101A5200E0936B02F0936C02B7DF10970895C0DF3A
:101A6200B3CFEA0FFB1FE0936B02F0936C02089571
:101A7200E0E0E0936202EFE0E0936302E09169024A
:101A8200F0916A02A1DFEA17FB07089579DF319628
:101A9200E0936B02F0936C020895A7DF71DFEA1BFB
:101AA200FB0BE0936B02F0936C020895E0916702E6
:101AB200EF5FE0936702A09167020895E0E0E09390
:101AC20067023093680271CFE3E0E09375020C94F1
:101AD2009B08EBB3E07FEBBBD89AE1E0E0937302A3
:101AE2000895A0917702AF5FA0937702A031089585
:101AF200E5E0E0937402E0E0E0937602E093BB025B
:101B02000895EA930E94080C11E00895E09375028B
:101B12000C949B08E091D402F091D5020895E091D3
:101B2200CD02EE0FE093CD02E091D902E0300895AC
:101B3200F0E0E054FD4F0895E12F1F5FF9CFF195DA
:101B4200E195F0400895EF2FFF27E7FDFFEF08959D
:101B5200EA17E1E009F0EE270895EA17E1E009F457
:101B6200EE270895EA17E1E008F0EE270895EA1754
:101B7200FB07E1E00CF0EE270895FA9FF02DEB9FB2
:101B8200F00DEA9FE02DF10D08951CD0F6DF0EF462
:101B9200D6DF08950024112490E1AA0FBB1F001C78
:101BA200111C0E1A1F0A18F40E0E1F1E01C0A1608E
:101BB2009A9599F7FD01D001089504D0EBDF0EF458
:101BC200BEDF0895E894F7FF02C0B9DF6894B7FF5B
:101BD20006C0A095B095119600F8039400FA0895F6
:101BE2001B2EBF2FF12D1A2EAE2FE12D0895E19954
:101BF200FECFFF93FFB7F894AEBBBFBBE09AEDB345
:101C0200FFBFFF910895E199FECF9FB7F894AEBB55
:101C1200BFBBE09A8DB3E81719F0EDBBE29AE19AE7
:101C22009FBF08955A934A933A932A931A930A9319
:101C320008955D814C813B812A8119810881089533
:00000001FF
